:100000008A110A120528000009000730990083169A
:100010000510851005118312F430A0000130A100F5
:100020009421FE202F20AC012C08053C031C2B281A
:10003000AD012D083B3C031C25280230A000A10186
:1000400094210130AD07031C19281F3083050130AE
:10005000AC07031C14281F3083050C282E28051418
:10006000F430A0000130A1009421C4207420742039
:100070007D2074207420AC012C08023C031C5828FD
:100080009720B220CD20D620C4208520A020852016
:10009000AD012D08023C031C52286B200130AD0736
:1000A000031C49281F3083050130AC07031C3C2882
:1000B0001F3083058E2074207420742074209030AB
:1000C000A0000130A100942105102C30A0000130C7
:1000D000A10094210800EF20EF20EF20DF20EF2087
:1000E000EF20DF20DF200800EF20EF20EF20EF20BF
:1000F000DF20EF20DF20DF200800A920BB20A9207F
:10010000BB20A920BB20A9200800EF20DF20EF2082
:10011000EF20DF20EF20DF20DF200800EF20DF20AE
:10012000DF20DF20DF20EF20DF20DF200800EF20AE
:10013000EF20DF20EF20EF20DF20DF20DF2008008E
:10014000EF20EF20DF20DF20EF20DF20DF20DF2087
:100150000800EF20EF20DF20EF20DF20EF20DF205E
:10016000DF200800EF20DF20DF20DF20EF20EF205E
:10017000DF20DF200800EF20DF20EF20DF20EF204E
:10018000DF20DF20DF200800EF20DF20DF20DF205E
:10019000DF20DF20DF20DF200800EF20DF20DF204E
:1001A000EF20DF20DF20DF20DF200800EF20EF201E
:1001B000EF20EF20DF20DF20DF20DF200800051503
:1001C000053084000230AA005730A0000130A100A1
:1001D0002030A2000030A300CF2105110800053017
:1001E00084000230AA008730A0000130A1001C303A
:1001F000A2000030A300CF21051108000514F4303F
:10020000A0000130A10094212F214D212F214D214B
:100210002F215B213A213A211D219030A00001308D
:10022000A100942105102C30A0000130A1009421E0
:10023000080082217121712108008221712182210F
:100240000800712182217121712108007121822110
:100250008221712108007121712182210800712100
:100260007121712182210800822182218221822133
:100270007121080021214D212B214D2134214D21B7
:1002800019214D2126214D2119215B21080005113D
:100290003C30A000A1019421080005113C30A000D1
:1002A000A10194213C30A000A10194213C30A00088
:1002B000A1019421080005113C30A000A101942166
:1002C0003C30A000A10194213C30A000A101942168
:1002D0003C30A000A10194213C30A000A101942158
:1002E00008000515053084000230AA00F330A00094
:1002F0000130A1003C30A2000030A300CF21051145
:10030000472108000515053084000230AA00F330AB
:10031000A0000130A100F030A2000030A300CF21E6
:100320000511472108009329A00803199F29A62138
:10033000A003000000000000000000009429A108B4
:1003400003190800A621A103A00394290C30A500DD
:10035000A50BA829000000001230A200A20BB529AD
:10036000B721B721000000000800B721AE290D30E9
:10037000A400A40BB929000008001030A802000155
:10038000031C013EA902031C0800C6290A30A8026A
:100390000001031C013EA902031C0800C6292A080B
:1003A00080042008A8002108A900BD210130A20274
:1003B000031CA3032A0980052008A8002108A9001E
:1003C000BD21A208031DCF29A308031DCF290800C2
:02400E00B401FB
:00000001FF
